:0200000480007A
:100000006F008004732F2034930F80006308FF0378
:10001000930F90006304FF03930FB0006300FF038E
:10002000130F000063040F0067000F00732F2034CC
:1000300063540F006F00400093E19153171F0000BD
:1000400023223FFC6FF09FFF93000000130100008C
:10005000930100001302000093020000130300004C
:100060009303000013040000930400001305000034
:10007000930500001306000093060000130700001C
:100080009307000013080000930800001309000004
:1000900093090000130A0000930A0000130B0000EC
:1000A000930B0000130C0000930C0000130D0000D4
:1000B000930D0000130E0000930E0000130F0000BC
:1000C000930F0000732540F16310050097020000B4
:1000D000938202017390523073500018970200000F
:1000E00093824202739052309B021000939252030B
:1000F0009382F2FF7390023B9302F0017390023AF5
:100100007350403097020000938242017390523046
:10011000735020307350303093010000970200007C
:10012000938282EE73905230130510001315F5017F
:10013000635C05000F00F00F930110009308D005D9
:10014000130500007300000093020000638A0200A0
:1001500073905210B7B200009B82921073902230BD
:100160007350003097020000938242017390123462
:10017000732540F17300203093000000130100004C
:100180003B87204093030000930120006316774AC9
:1001900093001000130110003B87204093030000E0
:1001A00093013000631A7748930030001301700008
:1001B0003B8720409303C0FF93014000631E7746B6
:1001C000930000003781FFFF3B872040B78300008A
:1001D0009301500063127746B700008013010000BE
:1001E0003B872040B703008093016000631677448B
:1001F000B70000803781FFFF3B872040B783008036
:1002000093017000631A7742930000003781000069
:100210001B01F1FF3B872040B783FFFF9B83130047
:1002200093018000631A7740B70000809B80F0FF45
:10023000130100003B872040B70300809B83F3FF3E
:1002400093019000631A773EB70000809B80F0FF17
:10025000378100001B01F1FF3B872040B783FF7F00
:100260009301A000631A773CB7000080378100003B
:100270001B01F1FF3B872040B783FF7F9B83130067
:100280009301B000631A773AB70000809B80F0FFBB
:100290003781FFFF3B872040B78300809B83F3FFBC
:1002A0009301C000631A7738930000001301F0FF38
:1002B0003B872040930310009301D000631E7736E4
:1002C0009300F0FF130110003B8720409303E0FFF1
:1002D0009301E000631277369300F0FF1301F0FF03
:1002E0003B872040930300009301F00063167734AE
:1002F0009300D0001301B000BB8020409303200086
:1003000093010001639A70329300E0001301B00082
:100310003B8120409303300093011001631E713034
:100320009300D000BB801040930300009301200194
:1003300063947030130200009300D0001301B000EA
:100340003B87204013030700130212009302200092
:10035000E31452FE9303200093013001631E732CBB
:10036000130200009300E0001301B0003B8720401F
:100370001300000013030700130212009302200071
:10038000E31252FE93033000930140016316732A77
:10039000130200009300F0001301B0003B872040DF
:1003A00013000000130000001303070013021200E3
:1003B00093022000E31052FE93034000930150018A
:1003C000631C7326130200009300D0001301B000D9
:1003D0003B8720401302120093022000E31652FED6
:1003E0009303200093016001631877241302000037
:1003F0009300E0001301B000130000003B87204091
:100400001302120093022000E31452FE9303300003
:100410009301700163127722130200009300F00031
:100420001301B00013000000130000003B872040C0
:100430001302120093022000E31252FE93034000C5
:1004400093018001631A771E130200009300D0000D
:10045000130000001301B0003B872040130212007C
:1004600093022000E31452FE9303200093019001B5
:100470006314771C130200009300E00013000000D7
:100480001301B000130000003B872040130212004C
:1004900093022000E31252FE930330009301A00167
:1004A000631C7718130200009300F0001300000093
:1004B000130000001301B0003B872040130212001C
:1004C00093022000E31252FE930340009301B00117
:1004D00063147716130200001301B0009300D000DC
:1004E0003B8720401302120093022000E31652FEC5
:1004F000930320009301C0016310771413020000DE
:100500001301B0009300E000130000003B8720407F
:100510001302120093022000E31452FE93033000F2
:100520009301D001631A7710130200001301B00089
:100530009300F00013000000130000003B872040F0
:100540001302120093022000E31252FE93034000B4
:100550009301E0016312770E130200001301B00053
:10056000130000009300D0003B87204013021200CC
:1005700093022000E31452FE930320009301F00144
:10058000631C770A130200001301B000130000007F
:100590009300E000130000003B872040130212008C
:1005A00093022000E31252FE9303300093010002F5
:1005B00063147708130200001301B0001300000059
:1005C000130000009300F0003B872040130212004C
:1005D00093022000E31252FE9303400093011002A5
:1005E000631C7704930010FF3B0110409303F0005D
:1005F0009301200263127104930000023B810040CA
:10060000930300029301300263187102BB000040A3
:100610009303000093014002639070029300000175
:100620001301E0013B80204093030000930150023E
:1006300063147000631030020F00F00F638001003C
:100640009391110093E111009308D00513850100E7
:10065000730000000F00F00F930110009308D00505
:100660001305000073000000731000C000000000BC
:0C0670000000000000000000000000007E
:1010000000000000000000000000000000000000E0
:1010100000000000000000000000000000000000D0
:1010200000000000000000000000000000000000C0
:1010300000000000000000000000000000000000B0
:081040000000000000000000A8
:040000058000000077
:00000001FF
